:040000008031D6284D
:100008007E14803120007F08F3000B1D6F2800004C
:1000180000008530200095000B11701FF01A16287B
:100028008D122B28701BF01E22280D128D1E1D28E4
:100038000D1620008D160D1A8D122C28701F2728DA
:1000480010308D068D12F01E2C2820308D060D12D2
:10005800033021004D02F43003194C0203184328E1
:100068000130CC070030CD3DF3304C060330031986
:100078004D06031D5B28B430200095005B28210045
:10008800CC01CD017115F01D51280130A8070030B1
:10009800A93D0030AA3D0030AB3D5508031956284C
:1000A8000130D502540803195B280130D402CA3044
:1000B80021005602031865280130F2007208D6079D
:1000C8006F28D601F114711C6B284030F006F01F20
:1000D8006F282030F0068B188B102000911EC9283D
:1000E80023001908F2007208F40020009112701A17
:1000F800C9287A08031D85280230F20072082100F9
:10010800D7007408F2007A08203E86000230870083
:10011800720881007A0303199F28B02833309A287F
:1001280097280A309A2804309A280230F200720878
:100138002100D700B0287408453A031997280C3ACB
:1001480003199728203A031995281C3A031994286B
:10015800023A0319922899280130F2007208FA0726
:1001680035307A06031DBB28FA012100D7012A3051
:100178007406031DC4287A0821005702031C701650
:1001880023009D1CC9281D121D162000121A1212C8
:10019800111B111391199111921992117308FF00F3
:1001A8007E1009008031D828F001F101FA01A03051
:1001B80084000030850048309D31E92580312030A9
:1001C8008400013085004D309D31E9258031A03013
:1001D80084000130850040309D31E9258031203090
:1001E80084000230850035309D31E9257E102000DD
:1001F8008331C62BF11C5D2AF1108C319E2480318D
:1002080000308D319E258031053021004F020318C2
:10021800112905304E02031C172990310220803124
:100228009D31E42580318631102680312100410836
:100238002000AE00210042082000AF002100430842
:100248002000B00021003E082000AB0021003F083C
:100258002000AC00210040082000AD0097314C2759
:10026800803120002B08BE002C08BF002D08C000DC
:100278000030BB007A30BC004430BD009631A32664
:10028800803120003B08CB003C08CC003D08CD0065
:100298009431ED24803120004E082200DC0020003B
:1002A8004D082200DB0020004C082200DA00200064
:1002B8004B082200D90000302000BB007A30BC0077
:1002C8004430BD000830513E860001308700403F71
:1002D800A300413FA400423FA500433FA6009F3131
:1002E8009C27803120002308BE002408BF00250871
:1002F800C0009631A326803120003B082100BB00B6
:1003080020003C082100BC0020003D082100BD0061
:10031800220056082302031D932955082202031CB4
:100328009C2901302000E60066082100D0079E299C
:100338002100D00100302000CB008230CC004230B8
:10034800CD00210032082000CE0021003308200013
:10035800CF00210034082000D000903111208031D6
:100368000318BD2901302000E60066082100D207E5
:10037800BF292100D201F01D202A22002E089E311B
:100388007426803120002308CB002408CC002508DF
:10039800CD0021003B082000CE0021003C082000B1
:1003A800CF0021003D082000D0009031112080317D
:1003B8000318E52901302000E60066082100D1076E
:1003C800E7292100D10100302000CB00C830CC0043
:1003D8004230CD00210041082000CE002100420813
:1003E8002000CF00210043082000D00090311120C8
:1003F800803103180F2A023022002C06031D072A19
:10040800893105218031033022002C06031D0F2A73
:100418008A31C522803120008D19562A3030F500E6
:100428007530F6009E310126803120008D19562A3C
:1004380090314D208031562A210053089E31742670
:10044800803120002308CB002408CC002508CD00EB
:1004580021003B082000CE0021003C082000CF00EE
:1004680021003D082000D000903111208031031870
:10047800442A01302000E60066082100D107462AF8
:100488002100D10120000D19562A3030F5007530B1
:10049800F6009E310126803120000D19562A94312C
:1004A800692480319131CA21803100308931E321BA
:1004B8008031711D08007111A03021009E000130AB
:1004C8009D000230F5000030F6009E310126803193
:1004D80021009D149D186E2A1C082000E600E701E3
:1004E80066082100E800200067082100E9000830BC
:1004F800E835E90D890B7C2A1B082000E600E70196
:1005080066082100E807200067082100E93D00305F
:100518002000AB00A030AC003B30AD0021006908E2
:100528002000A400210068082000A3009E3147266F
:10053800803120002308AE002408AF002508B00051
:1005480097314C27803120002B082100EA00200039
:100558002C082100EB0020002D082100EC006A087F
:100568002000AB0021006B082000AC0021006C08C3
:100578002000AD0021006A082000AE0021006B08B1
:100588002000AF0021006C082000B00097314C27F4
:10059800803120002B082100B20020002C08210007
:1005A800B30020002D082100B400C9302000AB00A2
:1005B8007230AC004130AD00210032082000AE009E
:1005C800210033082000AF00210034082000B000CB
:1005D80097314C27803120002B082100B2002000E1
:1005E8002C082100B30020002D082100B400320897
:1005F8002000BE00210033082000BF00210034087D
:100608002000C00021006A082000AE0021006B080D
:100618002000AF0021006C082000B000B330AB0010
:10062800A930AC004230AD0097314C278031200012
:100638002B08BB002C08BC002D08BD009D31F825F7
:10064800803120003B08C1003C08C2003D08C300BF
:100658008B31A823803120003E082100B200200001
:100668003F082100B300200040082100B4001F30DB
:100678002000BE000C30BF004330C000210032080B
:100688002000C100210033082000C20021003408E6
:100698002000C3008B31A823803120003E082100B0
:1006A800B20020003F082100B300200040082100CC
:1006B800B400F01D080024082000E60021002508E9
:1006C8002000E700210026082000E8002100270874
:1006D8002000E90021003E082000CB0021003F084F
:1006E8002000CC00210040082000CD009431ED24EA
:1006F800803120004B08EA004C08EB000030EB1B6F
:10070800FF30EC00ED006A08E6076B08E73D6C086F
:10071800E83D6D08E93D69082100A7002000680848
:100728002100A600200067082100A5002000660817
:100738002100A40022005908210020072000E6001B
:1007480022005A082100213D2000E70022005B0812
:100758002100223D2000E80022005C082100233D02
:100768002000E90069082100A30020006808210092
:10077800A200200067082100A100200066082100CF
:10078800A000080096310726833137309E315C2659
:100798008331003A0319F32BF50137309F312927AC
:1007A80083311030F5002730F6009E310126833161
:1007B8008831002083319E31AC2683311030F5001A
:1007C8002730F6009E310126833193316C23833123
:1007D8001030F5002730F6009E3101268331923122
:1007E800F522833188310020833192312A228331E6
:1007F80000302100B5000030B6000030B7000030EE
:10080800B8000030B9000030BA000030A70000304E
:10081800A6000030A5000030A4000030A30000307E
:10082800A2000030A1000030A0006400711D1A2C45
:1008380071116400711D1E2C71117013F016711066
:10084800F01300302100AB000030AA000030A900EE
:100858000030A8008030C8000030C900C601C701B8
:100868006400701E3A2C8E31B42683318031FE200C
:100878008331F01DE82D043022002C06031DD82CEE
:1008880021005408031DD82C22002F082300E00063
:1008980060082100D40000302000CB00A030CC003C
:1008A8004030CD000030BB007A30BC004430BD0081
:1008B800220025082000A400220024082000A3000C
:1008C8009E314726833120002308BE002408BF003C
:1008D8002508C0009631A326833120003B08CE00AE
:1008E8003C08CF003D08D000903111208331031C13
:1008F800822C00302000BE000030862C0030200002
:10090800BE008030BF003F30C00021003508200005
:10091800C100210036082000C2002100370820004D
:10092800C3008B31A823833120003E082100B50085
:1009380020003F082100B600200040082100B70031
:1009480000302000BB007A30BC004430BD002200DB
:1009580025082000A400220024082000A3009E31BE
:100968004726833120002308BE002408BF0025083D
:10097800C0009631A326833120003B08CB003C08F9
:10098800CC003D08CD00210035082000CE00210014
:1009980036082000CF00210037082000D000903111
:1009A80011208331031C701521005508031D292DC2
:1009B800FF304902FC30031948020318292DF016AC
:1009C800A0308600013087000430513E8400013099
:1009D800850004302300E00060080319F72C12009A
:1009E8001E00E00BF32C210049082000A200210082
:1009F80048082000A10004302300E000600820001F
:100A0800A3009F317327833104302100C8070030C9
:100A1800C93D0130C6070030C73D043022002C060E
:100A2800031D1A2D2100D501D50A212D22002F08DA
:100A38002300E00060082100D500D030F500073021
:100A4800F6009E3101268331F0122200300831046D
:100A580003194E2D30082300E0002200310823003E
:100A6800E100E201E301630821002B02031D4C2D84
:100A78002300620821002A02031D4C2D230061086F
:100A880021002902031D4C2D2300600821002802A3
:100A9800031870150430210052020318572D043032
:100AA8005102031C592D7015F01407304F0203181A
:100AB800612D07304E02031C632D7015F0140430AD
:100AC80050020318692D701D342CA03086000130A7
:100AD80087000430513E8400013085000430230033
:100AE800E000600803197C2D12001E00E00B782D31
:100AF800210049082000A200210048082000A10088
:100B080004302300E00060082000A3009F31732711
:100B18008331FF3021004902FC30031948020318D1
:100B28009D2D0430C8070030C93D0130C60700308C
:100B3800C73D8830F5001330F6009E310126833119
:100B4800FF302300E0006008A000FF30E0006008EC
:100B5800A100FF30E0006008A200FF30E00060085C
:100B6800A300210049082000A20021004808200015
:100B7800A10004302300E00060082000A3009F319A
:100B88007327833101302100C6070030C73DF011BB
:100B980070117013F016F01CD32D7114F01700307B
:100BA800B5000030B6000030B7000030B8000030A3
:100BB800B9000030BA000030AB000030AA000030A5
:100BC800A9000030A800342C043021005202031878
:100BD800F12D04305102031CFC2D0030B50000300B
:100BE800B6000030B700F0147013F0167114F01747
:100BF80007304F020318042E07304E02031C342C12
:100C08000030B5000030B6000030B700F0147013A3
:100C1800F0167114F017342C210037083604350407
:100C2800031D202E00302000DE000030DF000030E1
:100C3800E0009331E7230800210041082000CB00A1
:100C4800210042082000CC00210043082000CD00EC
:100C58000030CE00C830CF004230D0009031112093
:100C68008631031C080000302000BB007A30BC002D
:100C78004430BD0021003E082000BE0021003F088E
:100C88002000BF00210040082000C0009631A326A4
:100C9800863120003B08E3003C08E4003D08E500FD
:100CA8006308CB006408CC006508CD00D730BE00CF
:100CB800A330BF00BB30C000210035082000C100B0
:100CC800210036082000C200210037082000C30098
:100CD8008B31A823863120003E08CE003F08CF0084
:100CE8004008D0009031112086310318BB2ED73030
:100CF8002000CB00A330CC003C30CD0021003508CB
:100D08002000BE00210036082000BF00210037085F
:100D18002000C0006308BB006408BC006508BD0073
:100D28009D31F825863120003B08C1003C08C200EF
:100D38003D08C3008B31A823863120003E08CE0031
:100D48003F08CF004008D0009031112086310318A9
:100D5800B42ED7302000BE002330BF003C30222FF5
:100D6800D7302000BE002330BF003B30222FD730C1
:100D78002000BE00A330BF003B30C0002100350872
:100D88002000C100210036082000C20021003708D9
:100D98002000C3008B31A823863120003E08CB00F9
:100DA8003F08CC004008CD006308CE006408CF009F
:100DB8006508D00090311120863103183E2F20009D
:100DC8006308BE006408BF006508C000210035083C
:100DD8002000BB00210036082000BC002100370895
:100DE8002000BD009D31F825863120003B08C10058
:100DF8003C08C2003D08C3008B31A823863120007F
:100E08003E08CB003F08CC004008CD00D730CE00CC
:100E1800A330CF003C30D000903111208631031828
:100E28001C2FD7302000BE002330BF00BC30222F3B
:100E3800D7302000BE002330BF00BB30C0002100E7
:100E48002F082000C100210030082000C200210026
:100E580031082000C3008B31A823863120003E08CA
:100E68002100AF0020003F082100B000200040080A
:100E78002100B10021002F082000CB0021003008FC
:100E88002000CC00210031082000CD000030CE0029
:100E98000030CF00BF30D0009031112086310318C8
:100EA8005C2F00302100AF000030B000BF30B1002F
:100EB80000302000CB000030CC003F30CD002100B6
:100EC8002F082000CE00210030082000CF0021008C
:100ED80031082000D00090311120863103187B2F73
:100EE80000302100AF000030B0003F30B1002100D9
:100EF800310830042F04031908002F082000BE0011
:100F0800210030082000BF00210031082000C00067
:100F1800210035082000C100210036082000C20049
:100F2800210037082000C3008B31A8238631200018
:100F38003E08DE003F08DF004008E0009331E72369
:100F4800080000302000AB000030AA000030A900E3
:100F58000030A80023082204210420040319EF2FDD
:100F6800AC01AC0AA31BC42F0130A035A10DA20D02
:100F7800A30D890BB92F0130F5007508AC07B62F02
:100F88000130A835A90DAA0DAB0D890BC52F230873
:100F98002702031DD92F22082602031DD92F210855
:100FA8002502031DD92F20082402031CE42F200842
:100FB800A4022108A53B2208A63B2308A73B281426
:100FC8000130A336A20CA10CA00C890BE52F01302F
:100FD800AC02031DC42F2B08A3002A08A20029086D
:100FE800A1002808A0000800F50023009E1CF92F86
:060FF80075089A000800D4
:101000005430F50075082200B2006530F50075080F
:10101000B3007330F5007508B4007430F50075083E
:10102000B500B6010730F5007508AA00AB01AB0AA0
:10103000AC01AC0AC830A0000030A1008430A2008E
:101040000330A300C830A4000030A500AD01A60104
:10105000A701E830A8000330A900AE010530F50073
:101060007508AF00B001B101080002309F314C2774
:10107000883176082000D2007508D10004309F31F5
:101080004C27883176082000D0007508CF00220058
:101090006B082000CF0222006C082000D03B0630F5
:1010A0009F314C27883176082000D4007508D30082
:1010B00008309F314C27883176082000D60075080B
:1010C000D50022006B082000D50222006C08200009
:1010D000D63B51085204031D7A2891302100DE00CE
:1010E000AD30DF003E30E0000030E1002030E200B3
:1010F0004230012920004F09CB005009CC00CB0A17
:101100000319CC0A55084B07A30056084C3DA40010
:101110009E314726883120002308BB002408BC00EC
:101120002508BD005109CD005209CE00CD0A031992
:10113000CE0A53084D07A30054084E3DA4009E312B
:101140004726883120002308BE002408BF00250858
:10115000C0009631A326883120003B082100DE0024
:1011600020003C082100DF0020003D082100E000B5
:1011700020005608A4005508A3009E314726883158
:1011800020002308AE002408AF002508B000063078
:10119000D83E86008701403FAB00413FAC00423F54
:1011A000AD0097314C27883120002B08BB002C085C
:1011B000BC002D08BD009D31F825883120003B087A
:1011C000BE003C08BF003D08C0005408A4005308FE
:1011D000A3009E314726883120002308C10024083F
:1011E000C2002508C3008B31A823883120003E08A7
:1011F0002100E10020003F082100E200200040081B
:101200002100E3009E318F26080021003A083904AE
:1012100038040319080000302000BB007A30BC00FD
:101220004430BD00210041082000BE0021004208DA
:101230002000BF00210043082000C0009631A326F3
:10124000893120003B08E3003C08E4003D08E5004C
:101250006308BB006408BC006508BD0021003808B5
:101260002000BE00210039082000BF0021003A08FC
:101270002000C0009631A326893120003B082100C0
:10128000AC0020003C082100AD0020003D082100FA
:10129000AE0000302000BB007A30BC004430BD00FE
:1012A000220029082000A400220028082000A30012
:1012B0009E314726893120002308BE002408BF0044
:1012C0002508C0009631A326893120003B08CB00B9
:1012D0003C08CC003D08CD0021002C082000CE00A9
:1012E00021002D082000CF0021002E082000D00072
:1012F0009031112089310318A82900302000BB004B
:101300007A30BC004430BD00220029082000A4002F
:10131000220028082000A3009E31472689312000A2
:101320002308BE002408BF002508C0009631A3266C
:10133000893120003B082100AC0020003C0821003E
:10134000AD0020003D082100AE0070137114AC29DF
:10135000711CAC2971107017210037082E06031D6F
:10136000B72936082D06031DB72935082C060319A1
:1013700008002C08B5002D08B6002E08B7002F086D
:101380002000BE00210030082000BF0021003108ED
:101390002000C000210035082000C10021003608CF
:1013A0002000C200210037082000C3008B31A82391
:1013B000893120003E08DE003F08DF004008E000E1
:1013C0009331E72308002000DA0021002B082200D7
:1013D000D40021002A082200D3002100290822007D
:1013E000D200210028082200D1002100410820005D
:1013F000CB00210042082000CC002100430820003F
:10140000CD009431ED24893120004C082200D60013
:1014100020004B082200D50021003E082000CB0010
:1014200021003F082000CC00210040082000CD0012
:101430009431ED24893120004C082200D80020008E
:101440004B082200D70000302000A3000030A2008B
:101450000E30A1001030A000210027082000A700B6
:10146000210026082000A600210025082000A50054
:10147000210024082000A4008731A52789312000FD
:1014800023082200E000200022082200DF002000C4
:1014900021082200DE00200020082200DD000030AC
:1014A0002000A3000030A2000E30A1001030A000E8
:1014B000210023082000A700210022082000A60008
:1014C000210021082000A500210020082000A40000
:1014D0008731A5278931200023082200E40020005D
:1014E00022082200E300200021082200E200200060
:1014F00020082200E100210032082000CB0021005A
:1015000033082000CC00210034082000CD009431A5
:10151000ED24893120004C082200E60020004B0811
:101520002200E50057085804031D9A2A6C08EA00B7
:101530006B08E90020005A0803190800A030860053
:101540000130870051308400013085001C302000BC
:10155000D90059080319B02A12001E00D90BAC2A71
:101560002000DB011C305B02031808005B08A03E72
:1015700086000130870001088731F8278931013062
:101580002000D9005908DB07B22A220026082704C8
:101590000319080000302000BB007A30BC00443042
:1015A000BD00210041082000BE00210042082000AB
:1015B000BF00210043082000C0009631A3268A31D5
:1015C00020003B08E3003C08E4003D08E500220061
:1015D00027082000A400220026082000A3009E3136
:1015E00047268A3120002308BB002408BC002508B8
:1015F000BD006308BE006408BF006508C0009631E6
:10160000A3268A3120003B082100AC0020003C08C2
:101610002100AD0020003D082100AE000030200078
:10162000BB007A30BC004430BD00220029082000F5
:10163000A400220028082000A3009E3147268A31FA
:1016400020002308BE002408BF002508C0009631F2
:10165000A3268A3120003B08CB003C08CC003D0883
:10166000CD0021002C082000CE0021002D082000F4
:10167000CF0021002E082000D000903111208A31A7
:1016800003186D2B00302000BB007A30BC004430C2
:10169000BD00220029082000A40022002808200004
:1016A000A3009E3147268A3120002308BE0024086B
:1016B000BF002508C0009631A3268A3120003B08D0
:1016C0002100AC0020003C082100AD0020003D08B6
:1016D0002100AE0070137114712B711C712B7110ED
:1016E0007017210037082E06031D7C2B36082D06A7
:1016F000031D7C2B35082C06031908002C08B500A7
:101700002D08B6002E08B7002F082000BE002100CB
:1017100030082000BF00210031082000C000210057
:1017200035082000C100210036082000C200210039
:1017300037082000C3008B31A8238A3120003E08DF
:10174000DE003F08DF004008E0009331E723080097
:1017500020003E08C4003F08C5004008C600031032
:10176000450D460DC7004708CA004108C40042089D
:10177000C5004308C6000310450D460DC7004708C5
:10178000C9004A080319D02B49084A020318D72B6D
:101790004A03FF3A4907C40019304402031CD72BFF
:1017A0004108BE004208BF004308C00008004908C5
:1017B000031908004A0849020318E62B4903FF3AB7
:1017C0004A07C40019304402031808000630C40058
:1017D0004408C800C01BC817C31B4817BF17FF30F9
:1017E000BE05FF30BF050030C005C217FF30C10580
:1017F000FF30C2050030C30549084A020318222CF5
:101800000130C135C20DC30D890B012C0130C90255
:1018100049084A0603191D2C0130C8024808073937
:1018200003191D2C002C0130C036BF0CBE0C890BD7
:10183000142C0130C4004408CA074A084906031999
:10184000472C132C4A0849020318472C0130BE3597
:10185000BF0DC00D890B272C0130CA0249084A066A
:101860000319432C0130C802480807390319432CD7
:10187000262C0130C336C20CC10C890B3A2C013026
:10188000C4004408C9074A084906031D392CC81F6B
:10189000592CFF30BE06FF30BF06FF30C0060130B6
:1018A000BE07003003180130BF07003003180130B5
:1018B000C007481F6B2CFF30C106FF30C206FF3047
:1018C000C3060130C107003003180130C2070030E1
:1018D00003180130C307C8013E08C1073F08C23DD5
:1018E0004008C33DC31F862CFF30C106FF30C2062F
:1018F000FF30C3060130C107003003180130C207B2
:10190000003003180130C307C801C80A4108F500B8
:101910004208F6004308F7004A08C4004408F800EB
:101920004808C5004508F90092318E22750820004C
:10193000BE007608BF007708C00008009D31DF2593
:101940008C31D0309D31EF258C3118309D31EF2511
:101950008C319D31E4258C312000D90118302000D4
:1019600059060319D62C9D31DF258C31D1309D319C
:10197000EF258C3101309E31E7268C312000D400D8
:101980005408DB0001309E31E7268C312000D40062
:101990005408DA0000309E31E7268C312000D40054
:1019A0005408D9009D31E4258C31AE2C5B0A031D0F
:1019B000E22C5A0A031DE22C0130D4005408210005
:1019C000CF0708002100CF012000DB1FEB2C2200F5
:1019D000E701E801FE2C20005A08D400D5015B087D
:1019E000D600D7015608D700D60154085607220062
:1019F000E70020005508573D2200E800701C042D28
:101A00006735E700680DE8000330D83E860087019F
:101A1000403F2000BE00413FBF00423FC0002100C8
:101A200058082000AB00210059082000AC0021001C
:101A30005A082000AD00220068082000A4002200FF
:101A400067082000A3009E3147268C312000230820
:101A5000AE002408AF002508B00097314C278C3128
:101A600020002B08C1002C08C2002D08C3008B31B8
:101A7000A8238C3120003E082100C10020003F082F
:101A80002100C200200040082100C30041082000BE
:101A9000BE00210042082000BF00210043082000B2
:101AA000C00021003E082000AB0021003F082000BC
:101AB000AC00210040082000AD000C30D83E86006C
:101AC0008701403FAE00413FAF00423FB000973139
:101AD0004C278C3120002B08C1002C08C2002D0897
:101AE000C3008B31A8238C3120003E082100C100A7
:101AF00020003F082100C200200040082100C30050
:101B000041082000CB00210042082000CC00210029
:101B100043082000CD000030CE000030CF00003060
:101B2000D000903111208C310318080000302100C2
:101B3000C1000030C2000030C30008002000DA00FD
:101B40005A08031DB02D2100370836043504031D43
:101B5000B02D0030BE000030BF000030C0000800D3
:101B60009D31DF258D31D0309D31EF258D313830DD
:101B70009D31EF258D319D31E4258D312000D90136
:101B80003830200059060319E82D9D31DF258D31AD
:101B9000D1309D31EF258D3101309E31E7268D31D9
:101BA0002000D4005408DC0001309E31E7268D313E
:101BB0002000D4005408DB0000309E31E7268D3130
:101BC0002000D4005408D9009D31E4258D31C02D6A
:101BD0005C0A031DF42D5B0A031DF42D0130D400B3
:101BE00054082100CE0708002100CE012000DC1F90
:101BF000042E2200E901EA0100302100BE0000307D
:101C0000BF000030C000080020005B08D400D501F0
:101C10005C08D600D7015608D700D60154085607ED
:101C20002200E90020005508573D2200EA0020006C
:101C30005A080319202E22006A08EC006908EB00FC
:101C400022006C082000A40022006B082000A300E2
:101C50009E3147268D3120002308BB002408BC009C
:101C60002508BD009D31F8258D3120003B08BE00C0
:101C70003C08BF003D08C00022006A082000A40004
:101C8000220069082000A3009E3147268D312000E4
:101C90002308C1002408C2002508C3008B31A823F3
:101CA0008D3120003E082100BE0020003F082100A9
:101CB000BF00200040082100C0003E082000CB00EB
:101CC00021003F082000CC00210040082000CD006A
:101CD0000030CE000030CF000030D0009031112015
:101CE0008D3103187A2E00302100BE000030BF0075
:101CF0000030C0000930D83E86008701403F2000F8
:101D0000BE00413FBF00423FC00021003E0820000E
:101D1000AB0021003F082000AC002100400820005B
:101D2000AD000630D83E86008701403FAE00413FFF
:101D3000AF00423FB00097314C278D3120002B0877
:101D4000C1002C08C2002D08C3008B31A82320003D
:101D50003E082100BE0020003F082100BF002000F7
:101D600040082100C0000800243024002006031988
:101D7000C72FFD2FF019FD2F943169248E31FD2FCF
:101D8000F01DFD2F90314D208E31FD2FF019FD2FCC
:101D9000210046084704031DD02E903191208E313A
:101DA000210046088731F8278E3121004708873106
:101DB000F8278E31043022002C06031DE12E01305D
:101DC000E32E22002F088731F8278E319031D5205D
:101DD0008E31FD2FF019FD2F91311D218E31FD2FF8
:101DE000F019FD2F883135208E31FD2FF019FD2F90
:101DF000953174258E31FD2F883100208E319E3132
:101E0000AC268E311030F5002730F6009E310126C9
:101E10008E3193316C238E31FD2F203086000230BD
:101E20008700203084000130850031302000E3003D
:101E3000630803191F2F12001E00E30B1B2F9E3196
:101E40001F268E31FD2F20308600013087000230A2
:101E5000203E84000230850031302000E30063081A
:101E60000319362F12001E00E30B322F9E31AC26D1
:101E70008E311030F5002730F6009E3101268E316C
:101E800092312A228E31FD2F01308931E3218E31AA
:101E9000FD2F15308731F8278E31FD2F9E310C260E
:101EA0008E31FD2FF019FD2F02309F314C278E31DE
:101EB00076082100C5007508C40000302000BB0072
:101EC0007A30BC004430BD00210045082000A40049
:101ED000210044082000A3009E3147268E312000B7
:101EE0002308BE002408BF002508C0009631A326A1
:101EF0008E3120003B082100B50020003C08210065
:101F0000B60020003D082100B70035082000DE00A3
:101F1000210036082000DF00210037082000E00003
:101F20009331E7238E31FD2F240022082000E300A7
:101F3000E4016308A3006408A400A501A50A9F3179
:101F4000C6278E31230020088731F8278E31FD2FD8
:101F5000240023082000E30063082300A0002400DD
:101F600022082000E300E4016308A1006408A20045
:101F7000A301A30A9F3173278E311030F50027305B
:101F8000F6009E3101268E31FD2F0028FD2F240002
:101F90002108433A03194E2F063A0319A82F0C3A89
:101FA0000319522F1B3A0319FC2E013A0319C02EB4
:101FB000053A0319492F343A0319C52F063A031974
:101FC000C62E013A0319942F0C3A0319F02E053A44
:101FD0000319F62E1E3A03190D2F013A0319BA2ED2
:101FE000073A0319FD2F013A0319EA2E033A0319A0
:101FF000442F013A0319232FFD2F7012FA01080014
:1020040020008E150E1638302400950096010830F5
:1020140092002000911192112400941708002000CE
:10202400CD1F28284B09D1004C09D2004D09D300FB
:10203400D10A0319D20A0319D30A00305107CB007D
:102044000030523DCC008030533DCD00D01F3E289F
:102054004E09D1004F09D2005009D300D10A031907
:10206400D20A0319D30A00305107CE000030523D82
:10207400CF008030533DD0008030CD068030D00674
:1020840050084D02031D08004F084C02031D0800B0
:102094004E084B020800F0117013F01600302100B6
:1020A400B5000030B6000030B7000030B800003092
:1020B400B9000030BA000030AB000030AA00003094
:1020C400A9000030A800FF302000A6002608230045
:1020D400A000FF302000A60026082300A100FF3046
:1020E4002000A60026082300A200FF302000A6003E
:1020F40026082300A300210049082000A200210093
:1021040048082000A1000430A6002608A3009F313F
:10211400732701302100C6070030C73D0800803016
:102124002100C8000030C900C601C70149082000C9
:10213400A400210048082000A3000430A8002808B7
:10214400A5009F31C627903104302100C807003014
:10215400C93D0130C6070030C73D2000A901A90AC6
:10216400AA0104302A020318C7282A08A03E8600C0
:1021740001308700010A031DA9010130A8002808C5
:10218400AA0704302A02031CB72864002000290887
:10219400031D0800FF3021004902FB3003194802E7
:1021A40003180800982880302100C8000030C900B6
:1021B40049082000A400210048082000A30004309E
:1021C400A8002808A5009F31C627903104302100BB
:1021D400C8070030C93D2000A901A90AAA0104309A
:1021E4002A0203180F292A08A03E8600013087001E
:1021F40001088731F827903120002A08A03E860084
:1022040001308700010A031DA9010130A800280834
:10221400AA0704302A02031CF528640020002908B8
:10222400031D0800FF3021004902FB300319480256
:1022340003180800DA2802309F314C2791317608C0
:102244002100C5007508C40044084504031D302955
:102254004530D8008030D9003F3062292200680818
:102264002000A400220067082000A3009E31472616
:10227400913120002308BB002408BC002508BD00C0
:10228400210045082000A400210044082000A300E8
:102294009E314726913120002308BE002408BF0048
:1022A4002508C0009631A326913120003B08210067
:1022B400D80020003C082100D90020003D0821005E
:1022C400DA000030DB000030DC000030DD009E313D
:1022D4008F2608002000DD00C0295A08DC005908B8
:1022E400DB005C0DDC0CDB0C5C0DDC0CDB0C5B083C
:1022F4002500910020005A08DC005908DB005C0D21
:10230400DC0CDB0C5B1C8929250093168B2925002A
:1023140093122000591C9129250013169329250096
:10232400131221000E118E14080020005A08DC003C
:102334005908DB005C0DDC0CDB0C5C0DDC0CDB0CED
:102344005B082500980020005A08DC005908DB00CF
:102354005C0DDC0CDB0C5B1CB22925009A16B4293D
:1023640025009A122000591CBA2925001A16BC29E6
:1023740025001A1221000E158E10080020005D0899
:10238400013A03196F29033A03199729C929080047
:1023940000302000CB002030CC004230CD002100A2
:1023A40032082000CE00210033082000CF00210095
:1023B40034082000D0009031112091310318E6290F
:1023C400FF3026009800080021003B082000CB00C5
:1023D40021003C082000CC0021003D082000CD0055
:1023E4009431ED24913120004C08DA004B08D900D7
:1023F400D935DA0DD935DA0D5908203EDB00003025
:102404005A3DDC005C08803AD90080305902031D33
:102414000D2A40305B020318142A40302000DB00F0
:102424000030DC0020005C08803AD9008130590279
:10243400031D1E2A00305B02031C252AFF302000E6
:10244400DB000030DC0020005B0826009800080058
:1024540000302000A300A4003130A8002808A50003
:102464009F31C62792312030860001308700A0308A
:1024740084000130850031302000A80028080319A9
:10248400472A12001E00A80B432A0B3022002F02F9
:10249400031C522A05302000A80028082200AF009F
:1024A4002D082100530203185D2A53082000A800B8
:1024B40028082200AD0022002E08031D682A2100EE
:1024C40053082000A80028082200AE002508210097
:1024D4004B02031D712A2200240821004A0203181A
:1024E4007A2A4B082200A50021004A082200A400F1
:1024F4002200290821004B02031D842A22002808F7
:1025040021004A02031808004B082200A9002100F8
:102514004A082200A800080078080319962A7708B8
:1025240076047504031DA82A0030F5000030F60077
:102534000030F700080001302000A0002008F80750
:102544000130F736F60CF50C890BA32AFE3077051B
:102554000319C22A9D2A01302000A0002008F80790
:102564000130F507003003180130F6070030031876
:102574000130F7070130F736F60CF50C890BBD2A4C
:10258400FF3077050319CF2AAD2A0130F802013054
:10259400F535F60DF70D890BCA2AF61BD52A02303C
:1025A40078020318C72A7818DD2AFF30F5057F3032
:1025B400F605FF30F7050310F80C78082000A0009A
:1025C400A101A2011030A035A10DA20D890BE52AAD
:1025D4002008F5042108F6042208F70479080319F1
:1025E4000800F717080064302000A3000030A4009E
:1025F4001030A8002808A5009F31C6279231D83092
:1026040086008701A030840001308500103020004E
:10261400A80028080319122B12001E00A80B0E2B69
:1026240021005D085C045B0403191B2B93316C23AC
:1026340092317E302000A3000030A400A501A50A39
:102644009F31C6279231230020082000A800A90149
:1026540028082100CA00200029082100CB004B08CB
:10266400F6004A08F500E830F7000330F8009E3120
:10267400C926923176082100CB007508CA004A08A1
:102684004B0403194C2B3A304B02993003194A027C
:10269400031C502B1030CA002730CB007F302000A1
:1026A400A3000030A400A501A50A9F31C6279231DA
:1026B400230020082000A80028082100D300973018
:1026C4005302031C08006E302000A80028082100D3
:1026D400D300080045302100D8008030D9003F30B5
:1026E400DA000030DB000030DC000030DD00913027
:1026F400DE00AD30DF003E30E0000030E10020308D
:10270400E2004230E300D730E400A330E5003C307F
:10271400E600BE302000A60026082100E700A03015
:10272400860001308700D8308400850110302000F5
:10273400A60026080319A22B12001E00A60B9E2B2E
:1027440064302000A1000030A2001030A60026084A
:10275400A3009F31732793311030F5002730F60022
:102764009E310126933110302100CA002730CB005E
:102774000A302000A60026082300A0007E30200096
:10278400A1000030A200A301A30A9F317327933153
:102794001030F5002730F6009E31012693316E305B
:1027A4002000A60026082100D3006E302000A600D9
:1027B40026082300A0007F302000A1000030A200E2
:1027C400A301A30A9F317327080020005E08CB00F1
:1027D4005F08CC006008CD000030CE000030CF0090
:1027E4000030D0009031112093310318002C0030B8
:1027F4002000DE000030DF000030E00020005E0832
:10280400CB005F08CC006008CD000030CE008030E3
:10281400CF004030D00090311120933103183A2C6E
:10282400210067089E317426933120002308AE00EE
:102834002408AF002508B0005E08AB005F08AC00B8
:102844006008AD0097314C27933120002B08CB0052
:102854002C08CC002D08CD009431ED2493312000B8
:102864004C08DA004B08D900023091316C21080081
:10287400210067362000E100E2016108A30062083C
:10288400A4009F310727933120002308AE002408B9
:10289400AF002508B0005E08AB005F08AC0060081C
:1028A400AD0097314C27933120002B08CB002C0826
:1028B400CC002D08CD009431ED24933120004C0838
:1028C400DA004B08D900013091316C210800F01076
:1028D400F01570117110F0137017F0120030210010
:1028E400A7000030A6000030A5000030A40000308E
:1028F400A3000030A2000030A1000030A00000308E
:10290400AB000030AA000030A9000030A8008030DD
:10291400C8000030C900C601C70122002F082000EA
:10292400CB004B082100D500E12C00302000BB0077
:102934007A30BC004430BD00220025082000A400E9
:10294400220024082000A3009E3147269431200051
:102954002308BE002408BF002508C0009631A32622
:1029640020003B082100B50020003C082100B600EF
:1029740020003D082100B700080022002D089E31E8
:102984007426200023082100B80020002408210018
:10299400B900200025082100BA00080000302100F9
:1029A400B5000030B6000030B700D501D50A2200CA
:1029B4002F082000CB004B082100D400080022007F
:1029C4002C088400053004020318080098310435EB
:1029D400003E8200080020004B08CF004C08D000C5
:1029E4004D08D1000310500D510DD2005208D800EB
:1029F4005808031D062D0030CE000030CD000030F5
:102A0400CC000030CB0008004B08CF004C08D000AD
:102A14004D08D1001730D136D00CCF0C890B0D2DB9
:102A24004F08D2005208D300CC17FF30CB05FF303B
:102A3400CC050030CD054B08D4004C08D5004D081A
:102A4400D600D7018E30D802D81F442D5808803ABA
:102A54008F3E0318362D0030CE000030CD000030FC
:102A6400CC000030CB0008000130D736D60CD50C92
:102A7400D40C890B372D0130CF004F08D807031928
:102A84005D2D362D18305802031C5A2D0030CE000F
:102A94000030CD000030CC000030CB000800013005
:102AA400D435D50DD60DD70D890B522D0130D80252
:102AB4005808031D512D530803196B2DD409D5094A
:102AC400D609D709D40A0319D50A0319D60A031952
:102AD400D70A5708CE005608CD005508CC00540834
:102AE400CB00080000302100E4000030E500003095
:102AF400E6008C319E24953102309F314C2795316C
:102B040076082100C5007508C40041082000CB00E8
:102B1400210042082000CC00210043082000CD0001
:102B2400210045082000A400210044082000A3003F
:102B34009E314726953120002308CE002408CF007B
:102B44002508D0009031112095310318042E21005E
:102B540041082000BB00210042082000BC002100E5
:102B640043082000BD009D31F825953120003B0825
:102B7400BE003C08BF003D08C000210045082000FD
:102B8400A400210044082000A3009E31472695316B
:102B940020002308C1002408C2002508C3008B318B
:102BA400A823953120003E082100E40020003F08BE
:102BB4002100E500200040082100E6003E08200036
:102BC400BB0021003F082000BC0021004008200079
:102BD400BD000C30D83E86008701403FBE00413F17
:102BE400BF00423FC0009631A326953120003B0828
:102BF4002100E40020003C082100E50020003D08FD
:102C04002100E6009E318F26080020009E1321003B
:102C14001D10220091139313971398139A139B1367
:102C2400013023008C008D019D132F00911321008E
:102C34009915191699161917991019109913F53031
:102C44008C00CC308D00FF308E0020008C108C1551
:102C54000C1D2E2E70142F2E7010FF3021008C00AE
:102C640020008D018E01183021009700023095005C
:102C74000C3024008D0020001E1021009511151524
:102C840095101510A43023009E0090309D009F11D4
:102C940008309B0001309C00E0308B002030210084
:102CA4009100FF3020009B000C30250093000C3075
:102CB4009A000C3026009A0025009E010430200062
:102CC4009C00260098019031022096319D31E42524
:102CD400963124001614F430F5000130F6009E31CC
:102CE4000126963124001615F430F5000130F60063
:102CF4009E31012696317013F0167114F0170030CE
:102D04002000DE000030DF000030E0009331E723D4
:102D140096312000E4010A306402031808000130EF
:102D24008D319E2596316030F500EA30F6009E31F3
:102D340001269631640001302000E3006308E407B3
:102D44008D2E20003E08C1003F08C2004008C30089
:102D54000310420D430DC4004408C9004908031D73
:102D6400BA2E0030BB000030BC000030BD000800AB
:102D74003B08C1003C08C2003D08C3000310420DDB
:102D8400430DC4004408CA004A08031DD02E003075
:102D9400BB000030BC000030BD0008000030C6009D
:102DA4000030C7000030C80089304A07C10041081C
:102DB400C9023E08C1003F08C2004008C3001030E9
:102DC400C336C20CC10C890BE22E4108C40044086E
:102DD400CA003B08C1003C08C2003D08C3001030D3
:102DE400C336C20CC10C890BF22E4108C40044083E
:102DF400CA068030C1004108CA05BF17FF30BE05AE
:102E0400FF30BF050030C005BC17FF30BB05FF30E5
:102E1400BC050030BD051830C1004108C5000130B3
:102E2400C635C70DC80D890B122F3D084002031D7E
:102E3400212F3C083F02031D212F3B083E02031CA7
:102E44002A2F3B08BE023C08BF3B3D08C03B46144A
:102E54000130BE35BF0DC00D890B2B2F0130C502CB
:102E6400031D112F4608F5004708F6004808F7002F
:102E74004908C1004108F8004A08C2004208F900A4
:102E840092318E2275082000BB007608BC007708BA
:102E9400BD00080020002B08B1002C08B2002D084A
:102EA400B3000310320D330DB4003408B5003508F7
:102EB400031D632F0030AB000030AC000030AD00C8
:102EC40008002E08B1002F08B2003008B300031028
:102ED400320D330DB4003408BA003A08031D792FBB
:102EE4000030AB000030AC000030AD0008003A0800
:102EF4007B3EB1003108B5072B08B1002C08B200A5
:102F04002D08B3001030B336B20CB10C890B852FE9
:102F14003108B4003408BA002E08B1002F08B200FA
:102F24003008B3001030B336B20CB10C890B952FB6
:102F34003108B4003408BA068030B1003108BA054B
:102F4400AC17AF17FF30AE05FF30AF050030B0054A
:102F54000030B6000030B7000030B8000730B100D0
:102F64003108B9002B1CBC2F2E08B6072F08B73D1B
:102F74003008B83D0130AD36AC0CAB0C890BBD2F1D
:102F84000130AE35AF0DB00D890BC32F0130B9023E
:102F9400031DB42F0930B1003108B9002B1CD82F00
:102FA4002E08B6072F08B73D3008B83D0130AD36BE
:102FB400AC0CAB0C890BD92F0130B836B70CB60C5E
:102FC400890BDF2F0130B902031DD02F3608F5001D
:102FD4003708F6003808F7003508B1003108F80062
:102FE4003A08B2003208F90092318E2275082000A6
:102FF400AB007608AC007708AD0008009431EC2CE7
:103004009431972C9431BF2C9431EC2C9431D02CE6
:103BBE009E3132262400161408009E31322624002F
:103BCE0016150800640080010131890BEA2D0034BE
:103BDE002000A0009E3132262000200824009100F3
:103BEE00080020003D083C043B0403190800803007
:103BFE00BD0608000130F5020030F63B750A031DC4
:103C0E00012E760A03190800012E2000A00138307B
:103C1E0020020318080020089E315C269E31873151
:103C2E00F8279E310130F90079082000A0070E2EEA
:103C3E00F70131307702031808007708203E86001E
:103C4E000230870001088731F8279E310130F600D7
:103C5E007608F707202E03102400141903140030E1
:103C6E00093DF500F6011F301605F70075087704BB
:103C7E00F8007608F9007808790403190800322E46
:103C8E0020002308F5002408F600F7018E30A60068
:103C9E002608F800F90192318E2275082000A30043
:103CAE007608A4007708A5000800F8006400230039
:103CBE0095185D2E7808F500F601750891007608C6
:103CCE0092003F30F700770895051514031015186C
:103CDE0003140030093D130808002000AA002A082A
:103CEE00A600A701A8012608F5002708F600280857
:103CFE00F7008E30A9002908F800F90192318E22C2
:103D0E0075082000A3007608A4007708A500080017
:103D1E00A030860001308700D83084008501103035
:103D2E002000A60026080319A02E12001E00A60BC6
:103D3E009C2E64302000A1000030A2001030A6009E
:103D4E002608A3009F3173270800A030860001309B
:103D5E008700203084000130850031302000A6001D
:103D6E0026080319BE2E12001E00A60BBA2E003016
:103D7E002000A100A2003130A6002608A3009F312A
:103D8E00732708002000A001A101751CD32E77080F
:103D9E002000A0077808A13D0130F735F80D890BFA
:103DAE00D42E0130F636F50C890BD92E7508760413
:103DBE00031DCC2E20002108F6002008F500080077
:103DCE002000A1009E3132269E31240096159E3190
:103DDE0032269E31240011082000A0002008A200E7
:103DEE009E3132269E31200021080319012F240016
:103DFE009612032F2400961616162000220808008D
:103E0E002000A801A41F122FA309A409A30A0319B5
:103E1E00A40AA801A80A2308F5002408F600F70151
:103E2E008E30A6002608F8002808A7002708F900FB
:103E3E0092318E2275082000A3007608A400770820
:103E4E00A5000800F800230095182A2F7808F60020
:103E5E00F7017608910077089200750893003F30BD
:103E6E00F60076089505200003108B1B03148B13A8
:103E7E002300151555309600AA309600951415118D
:103E8E002000031C08008B1708002000A00020084B
:103E9E00203E8600023087000108F700F8017708FF
:103EAE00A1007808A2002108F800F7017708A10008
:103EBE007808A2002008013E203E860002308700CE
:103ECE0001082107A10022080318220AA2002208D5
:103EDE00F6002108F50008009D31DF259F31AE3038
:103EEE009D31EF259F31200022089D31EF259F3116
:103EFE00200021089D31EF259F312000A5012308C8
:103F0E0025020318992F2508A03E86000130870050
:103F1E0001089D31EF259F3101302000A4002408B7
:103F2E00A507862F9D31E42508008E302000A700BE
:103F3E002708A800FF3026050319B12F0130A63639
:103F4E00A50CA40CA30C890BA62F0130A7002708E3
:103F5E00A807A12F2308F5002408F6002508F7006E
:103F6E002808A7002708F800F90192318E2275085B
:103F7E002000A3007608A4007708A50008009D3154
:103F8E00DF259F31AE309D31EF259F312000240873
:103F9E009D31EF259F31200023089D31EF259F3164
:103FAE009D31E4259F319D31DF259F31AF309D310D
:103FBE00EF259F312000A701250827020318F92FAE
:103FCE0001309E31E7269F312000A6002708A03E33
:103FDE00860001308700260881000130A6002608E1
:103FEE00A707E32F00309E31E7269F319D31E42550
:023FFE000800B9
:020000040001F9
:04000E001ACEDFDA4D
:10E0000041004100540069005300200041006B00B2
:10E010006B00750074006500730074006500720089
:10E020002000410053003900310037002000560025
:10E0300031002E0035002000300039002F00320062
:10E04000300032003000200043006F007000790083
:10E0500072006900670068007400200044004C00F2
:10E060003300480052005400000000000000FF0090
:00000001FF
